:020000040000FA
:04080000E7EF07F027
:1008100003B213EF05F0F2B42EEF05F09EB036EF01
:1008200005F09EB23EEF05F0F2A81AEF04F0F2B226
:1008300025EF04F0F2A620EF04F0F2B022EF04F06E
:1008400096EF07F0F296F290FF00CD90F2929EA004
:100850002FEF04F00101533F2FEF04F0542BAEC1F2
:10086000B2F1AFC1B3F1B0C1B4F1B1C1B5F1AAC138
:10087000AEF1ABC1AFF1ACC1B0F1ADC1B1F1A6C148
:10088000AAF1A7C1ABF1A8C1ACF1A9C1ADF1A2C158
:10089000A6F1A3C1A7F1A4C1A8F1A5C1A9F19EC168
:1008A000A2F19FC1A3F1A0C1A4F1A1C1A5F19AC178
:1008B0009EF19BC19FF19CC1A0F19DC1A1F196C188
:1008C0009AF197C19BF198C19CF199C19DF1CECF4E
:1008D00096F1CFCF97F153C198F154C199F1CF6AF6
:1008E000CE6A0101536B546B9E90CD800FBC0F8E6E
:1008F0000FBA7EEF04F00F8A96EF07F00F8C0FBE51
:10090000BAEF04F096C19AF197C19BF198C19CF19E
:1009100099C19DF19AC19EF19BC19FF19CC1A0F12B
:100920009DC1A1F19EC1A2F19FC1A3F1A0C1A4F1FB
:10093000A1C1A5F1A2C1A6F1A3C1A7F1A4C1A8F1CB
:10094000A5C1A9F1A6C1AAF1A7C1ABF1A8C1ACF19B
:10095000A9C1ADF1AAC1AEF1ABC1AFF1ACC1B0F16B
:10096000ADC1B1F1AEC1B2F1AFC1B3F1B0C1B4F13B
:10097000B1C1B5F101015E6B5F6B606B616B96514C
:100980005E2797515F2398516023995161239A51B3
:100990005E279B515F239C5160239D5161239E5193
:1009A0005E279F515F23A0516023A1516123A25173
:1009B0005E27A3515F23A4516023A5516123A65153
:1009C0005E27A7515F23A8516023A9516123AA5133
:1009D0005E27AB515F23AC516023AD516123AE5113
:1009E0005E27AF515F23B0516023B1516123B251F3
:1009F0005E27B3515F23B4516023B5516123D89072
:100A00000101613360335F335E33D890010161339C
:100A100060335F335E33D8900101613360335F33FD
:100A20005E3396EF07F00392030103EE00F080516E
:100A30007F0BE92604C0EFFF802B8151805D700B96
:100A4000D8A48B8200008051815D700BD8A48B925A
:100A500081518019D8B4079096EF07F0F294010104
:100A6000453F96EF07F0462B96EF07F09E90010169
:100A7000533F96EF07F0542B96EF07F09E92040039
:100A800062A143EF05F0077C07AC5EEF05F0C2748E
:100A9000C2B458EF05F0C3CFB3F5C4CFB4F5050128
:100AA000D890B433B333D890B433B3335FEF05F099
:100AB000C3CF55F1C4CF56F15FEF05F0C28207B442
:100AC000CCEF05F047C14BF148C14CF149C14DF1A4
:100AD0004AC14EF15EC162F15FC163F160C164F170
:100AE00061C165F196C1B6F197C1B7F198C1B8F18E
:100AF00099C1B9F19AC1BAF19BC1BBF19CC1BCF1DA
:100B00009DC1BDF19EC1BEF19FC1BFF1A0C1C0F1A9
:100B1000A1C1C1F1A2C1C2F1A3C1C3F1A4C1C4F179
:100B2000A5C1C5F1A6C1C6F1A7C1C7F1A8C1C8F149
:100B3000A9C1C9F1AAC1CAF1ABC1CBF1ACC1CCF119
:100B4000ADC1CDF1AEC1CEF1AFC1CFF1B0C1D0F1E9
:100B5000B1C1D1F1B2C1D2F1B3C1D3F1B4C1D4F1B9
:100B6000B5C1D5F1B3C5B5F5B4C5B6F5B5C5B7F5DD
:100B7000B6C5B8F5010155515B2756515C23E86AAB
:100B80005D230E2ECCEF05F05CC157F15DC158F12D
:100B90005B6B5C6B5D6B078E0201002F96EF07F0BD
:100BA0003C0E006F00C10CF101C10DF102C10EF14C
:100BB00003C10FF104C110F105C111F106C112F119
:100BC00007C113F108C114F109C115F10AC116F1E9
:100BD0000BC117F134C135F105012F51000AD8B40A
:100BE00095EF06F005012F51010AD8B41FEF06F06A
:100BF00005012F51020AD8B460EF06F005012F510C
:100C0000030AD8B460EF06F005012F51040AD8B4E6
:100C100060EF06F005012F51050AD8B460EF06F029
:100C200005012F51060AD8B460EF06F005012F51D7
:100C3000070AD8B460EF06F02F6B95EF06F00501B8
:100C400053672AEF06F054672AEF06F055672AEF3C
:100C500006F056672EEF06F095EF06F057C500F147
:100C600058C501F159C502F15AC503F10101010E40
:100C7000046F000E056F000E066F000E076F86EC06
:100C80001EF000C157F501C158F502C159F503C165
:100C90005AF5006753EF06F0016753EF06F002675D
:100CA00053EF06F0036795EF06F053C557F554C5AB
:100CB00058F555C559F556C55AF50F8895EF06F004
:100CC0000501306766EF06F095EF06F00FBE7BEF8B
:100CD00006F010A080EF06F00101476777EF06F0FD
:100CE000486777EF06F0496777EF06F04A677BEFD2
:100CF00006F080EF06F007AE80EF06F092EF06F008
:100D00000501312F95EF06F03C0E316F302F95EF36
:100D100006F00101000E626FE00E636FA50E646FB6
:100D2000010E656F0501306B0F880501626B33B7EB
:100D30009BEF06F062810CC100F10DC101F10EC103
:100D400002F10FC103F110C104F111C105F112C18B
:100D500006F113C107F114C108F115C109F116C15B
:100D60000AF117C10BF135C134F100C10CF101C119
:100D70000DF102C10EF103C10FF104C110F105C163
:100D800011F106C112F107C113F108C114F109C133
:100D900015F10AC116F10BC117F134C135F101018A
:100DA0008A67DAEF06F08B67DAEF06F08C67DAEF26
:100DB00006F08D67DEEF06F00EEF07F08EC100F152
:100DC0008FC101F190C102F191C103F10101010E46
:100DD000046F000E056F000E066F000E076F86ECA5
:100DE0001EF000C18EF101C18FF102C190F103C16B
:100DF00091F1006703EF07F0016703EF07F0026767
:100E000003EF07F003670EEF07F08AC18EF18BC185
:100E10008FF18CC190F18DC191F10F80D57ED5BE3F
:100E200069D0D6CF47F1D7CF48F145C149F1E86A3B
:100E3000E8CF4AF1109047C100F148C101F149C122
:100E400002F14AC103F101010A0E046F000E056FA1
:100E5000000E066F000E076F86EC1EF003AF1080C9
:100E6000010154A740EF07F00F9A0F9C0F9E01015C
:100E7000000E5E6F600E5F6F3D0E606F080E616F5B
:100E8000010147BF50EF07F0486750EF07F049678F
:100E900050EF07F04A6750EF07F0F28875EF07F060
:100EA000F2985E6B5F6B606B616B966B976B986B88
:100EB000996B9A6B9B6B9C6B9D6B9E6B9F6BA06BF6
:100EC000A16BA26BA36BA46BA56BA66BA76BA86BA6
:100ED000A96BAA6BAB6BAC6BAD6BAE6BAF6BB06B56
:100EE000B16BB26BB36BB46BB56BD76AD66A0101E9
:100EF000456B466B0CC100F10DC101F10EC102F151
:100F00000FC103F110C104F111C105F112C106F1C5
:100F100013C107F114C108F115C109F116C10AF195
:100F200017C10BF135C134F196EF07F002C0E0FFB5
:100F3000005001C0D8FF1000A6B29CEF07F00CC013
:100F4000A9FF0BC0A8FFA69EA69CA684F29E550EE4
:100F5000A76EAA0EA76EA682F28EA694A6B2AEEFD8
:100F600007F00C2A1200A96EA69EA69CA680A85087
:100F70000C2A120004012C0E826FA1EC0AF081EC05
:100F80001FF00C50B3EC07F0E8CF00F10C50B3ECBD
:100F900007F0E8CF01F101AFD3EF07F00101FF0E39
:100FA000026FFF0E036F24EC1FF02967DFEF07F0DD
:100FB0000401200E826FA1EC0AF0E4EF07F00401B7
:100FC0002D0E826FA1EC0AF04EEC1DF01200076AA4
:100FD0000F6A106A0F010D0EC16E860EC06E030EF1
:100FE000C26E0F01680E896E130E926E080E8A6E25
:100FF000F30E936E8B6A900E946EF18EF19E0E6AD4
:1010000001015B6B5C6B5D6B576B586BF29A010176
:10101000476B486B496B4A6B4B6B4C6B4D6B4E6B24
:101020004F6B506B516B526B456B466BD76AD66AF0
:101030000F01280ED56EF28A9D90B00ECD6E010183
:101040005E6B5F6B606B616B626B636B646B656B3C
:10105000666B676B686B696B536B546BCF6ACE6A58
:101060000F9A0F9C0F9E9D80760ECA6E9D82020184
:101070003C0E006FCC6A160EB3EC07F0E8CF00F11F
:10108000170EB3EC07F0E8CF01F1180EB3EC07F040
:10109000E8CF02F1190EB3EC07F0E8CF03F101013C
:1010A00003AF6DEF08F081EC1FF0160E0C6E00C15F
:1010B0000BF09CEC07F0170E0C6E01C10BF09CECD2
:1010C00007F0180E0C6E02C10BF09CEC07F0190E25
:1010D0000C6E03C10BF09CEC07F000C18AF101C15A
:1010E0008BF102C18CF103C18DF100C18EF101C100
:1010F0008FF102C190F103C191F11A0EB3EC07F028
:10110000E8CF00F11B0EB3EC07F0E8CF01F11C0EA5
:10111000B3EC07F0E8CF02F11D0EB3EC07F0E8CF17
:1011200003F1010103AFC3EF08F081EC1FF01A0EC9
:101130000C6E00C10BF09CEC07F01B0E0C6E01C195
:101140000BF09CEC07F01C0E0C6E02C10BF09CEC3B
:1011500007F01D0E0C6E03C10BF09CEC07F01A0E8D
:10116000B3EC07F0E8CF00F11B0EB3EC07F0E8CFCB
:1011700001F11C0EB3EC07F0E8CF02F11D0EB3EC49
:1011800007F0E8CF03F100C192F101C193F102C170
:1011900094F103C195F1240EAC6E900EAB6E240E4B
:1011A000AC6E080EB86E000EB06E1F0EAF6E04016E
:1011B000806B816B0F01900EAB6E0F019D8A030156
:1011C000806B816BC26B8B92C5EC24F0C5EC24F074
:1011D00021EC26F0A6EC22F0200EB3EC07F0E8CFCD
:1011E0002FF505012F51FF0AD8A4FEEF08F02F6B51
:1011F000200E0C6E2FC50BF09CEC07F00501010EC4
:10120000306F3C0E316F250EB3EC07F0E8CF00F1E4
:10121000260EB3EC07F0E8CF01F1270EB3EC07F090
:10122000E8CF02F1280EB3EC07F0E8CF03F101019B
:1012300003AF35EF09F081EC1FF0250E0C6E00C1F5
:101240000BF09CEC07F0260E0C6E01C10BF09CEC31
:1012500007F0270E0C6E02C10BF09CEC07F0280E75
:101260000C6E03C10BF09CEC07F000C153F501C1FB
:1012700054F502C155F503C156F500C157F501C13A
:1012800058F502C159F503C15AF5290EB3EC07F020
:10129000E8CF5BF505015C515B5DD8A05BC55CF5F3
:1012A00005012F51020A0EE181B862EF09F0050134
:1012B0005C2F5FEF09F05BC55CF562EF09F081BA66
:1012C00060EF26F0210EB3EC07F0E8CF00F1220E1C
:1012D000B3EC07F0E8CF01F1230EB3EC07F0E8CF51
:1012E00002F1240EB3EC07F0E8CF03F1010103AFE4
:1012F000A8EF09F081EC1FF0210E0C6E00C10BF07D
:101300009CEC07F0220E0C6E01C10BF09CEC07F078
:10131000230E0C6E02C10BF09CEC07F0240E0C6E39
:1013200003C10BF09CEC07F0210EB3EC07F0E8CF03
:1013300000F1220EB3EC07F0E8CF01F1230EB3EC7D
:1013400007F0E8CF02F1240EB3EC07F0E8CF03F189
:1013500000C15DF501C15EF502C15FF503C160F535
:10136000DDEC21F09FEC20F0EFEC1FF005012F5198
:10137000030A12E005012F51040A1DE005012F5157
:10138000050A24E005012F51060A32E005012F511C
:10139000070A38E00BEF0AF0ACC500F101010F0EAF
:1013A000001701010051000A36E001010051050A51
:1013B00032E008EF0AF0ACC500F101010F0E001792
:1013C00001010051000A27E008EF0AF00501AC51C5
:1013D000000A21E00501AC51150A1DE00501AC51E0
:1013E000300A19E00501AC51450A15E008EF0AF092
:1013F0000501AC51000A0FE00501AC51300A0BE0C9
:1014000008EF0AF00501AC51000A05E008EF0AF008
:1014100081BA60EF26F007900001F28EF28C07B0DF
:10142000CFEF1BF00FB0B0EF16F00FB874EF10F065
:101430000301805181197F0BD8B4CFEF1BF013EE5D
:1014400000F081517F0BE126812BE7CFE8FFE00B15
:10145000D8B4CFEF1BF023EE82F0C2513F0BD92658
:10146000E7CFDFFFC22BDF50780AD8A4CFEF1BF005
:1014700007808EC100F18FC101F190C102F191C1CD
:1014800003F10101040E046F000E056F000E066FDC
:10149000000E076F86EC1EF000AF58EF0AF0010156
:1014A000030E8E6F000E8F6F000E906F000E916F07
:1014B00003018251720AD8B4B0EF16F08251520A79
:1014C000D8B4B0EF16F08251750AD8B4B0EF16F068
:1014D0008251630AD8B48BEF18F08251690AD8B4EC
:1014E0006BEF13F082517A0AD8B47EEF14F0825178
:1014F000490AD8B40AEF13F08251500AD8B428EF41
:1015000012F08251700AD8B46BEF12F08251540A73
:10151000D8B496EF12F08251740AD8B4DCEF12F00E
:101520008251730AD8B4E0EF15F08251530AD8B44F
:1015300045EF16F082514C0AD8B4B5EF0AF0C0EF6F
:1015400018F0040114EE00F080517F0BE12682C4F4
:10155000E7FF802B120004010D0E826FA1EC0AF050
:101560000A0E826FA1EC0AF0120003018351300AC7
:10157000D8B476EF0DF003018351310AD8B482EF6D
:101580000EF003018351320AD8B4EEEF0EF00301DE
:101590008351330AD8B4FCEF0EF003018351340AAF
:1015A000D8B40AEF0FF003018351350AD8B479EFAC
:1015B00010F003018351360AD8B4A7EF10F00301ED
:1015C0008351460AD8B4CDEF0FF0030183514D0A81
:1015D000D8B4EFEF0BF0030183516D0AD8B409EFD3
:1015E0000CF0030183515A0AD8B4FCEF0DF003014B
:1015F0008351490AD8B4A7EF11F003018351500A6F
:10160000D8B4D9EF10F003018351540AD8B452EF83
:1016100011F003018351630AD8B429EF0CF00301E0
:101620008351430AD8B421EF0DF003018351730AAB
:10163000D8B427EF0CF003018351610AD8B43CEF12
:101640000BF003018351650AD8B4C4EF0DF0030118
:101650008351450AD8B4D2EF0DF003018351620AD9
:10166000D8B4E0EF0DF003018351420AD8B4EEEF95
:101670000DF0D8A4C0EF18F004014C0E826FA1EC5D
:101680000AF00401610E826FA1EC0AF09FEC20F0D9
:1016900004012C0E826FA1EC0AF081EC1FF0ABC5A7
:1016A00000F1010124EC1FF031C182F40401300E7D
:1016B0008227A1EC0AF032C182F40401300E8227A5
:1016C000A1EC0AF033C182F40401300E8227A1ECB0
:1016D0000AF004012C0E826FA1EC0AF081EC1FF0DD
:1016E000ACC500F1010124EC1FF031C182F404010A
:1016F000300E8227A1EC0AF032C182F40401300ED0
:101700008227A1EC0AF033C182F40401300E822753
:10171000A1EC0AF004012C0E826FA1EC0AF081EC1E
:101720001FF0ADC500F1010124EC1FF031C182F4BE
:101730000401300E8227A1EC0AF032C182F40401C8
:10174000300E8227A1EC0AF033C182F40401300E7E
:101750008227A1EC0AF004012C0E826FA1EC0AF0A2
:1017600081EC1FF0AEC500F1010124EC1FF031C186
:1017700082F40401300E8227A1EC0AF032C182F417
:101780000401300E8227A1EC0AF033C182F4040177
:10179000300E8227A1EC0AF004012C0E826FA1EC1E
:1017A0000AF081EC1FF0B3C500F1010124EC1FF039
:1017B00031C182F40401300E8227A1EC0AF032C15B
:1017C00082F40401300E8227A1EC0AF033C182F4C6
:1017D0000401300E8227A1EC0AF0D5EF10F0C2EC24
:1017E0001FF084C333F1CFEC1FF046EC1FF0200E46
:1017F0000C6E00C10BF09CEC07F000C12FF5050149
:101800002F51000A06E005012F51010A02E045ECC4
:1018100021F004014C0E826FA1EC0AF004014D0E80
:10182000826FA1EC0AF004012C0E826FA1EC0AF089
:1018300081EC1FF02FC500F124EC1FF033C182F4BE
:101840000401300E8227A1EC0AF0D5EF10F060EF12
:1018500026F004014C0E826FA1EC0AF00401630E25
:10186000826FA1EC0AF0EFEC1FF004012C0E826FE6
:10187000A1EC0AF03EEC0CF0D5EF10F081EC1FF07B
:10188000B1C500F10101003B0F0E001724EC1FF061
:1018900033C182F40401300E8227A1EC0AF0B1C5F5
:1018A00000F101010F0E0101001724EC1FF033C1FC
:1018B00082F40401300E8227A1EC0AF004012D0EFF
:1018C000826FA1EC0AF0B0C500F10101003B0F0EE0
:1018D000001724EC1FF033C182F40401300E82277C
:1018E000A1EC0AF0B0C500F101010F0E01010017D3
:1018F00024EC1FF033C182F40401300E8227A1ECE6
:101900000AF004012D0E826FA1EC0AF0AFC500F1C0
:101910000101003B0F0E001724EC1FF033C182F4CD
:101920000401300E8227A1EC0AF0AFC500F10101DD
:101930000F0E0101001724EC1FF033C182F40401E3
:10194000300E8227A1EC0AF00401200E826FA1EC78
:101950000AF0AEC500F10F0E0101001724EC1FF0D4
:1019600033C182F40401300E8227A1EC0AF0040195
:10197000200E826FA1EC0AF0ADC500F1010101015A
:10198000003B0F0E001724EC1FF033C182F404015A
:10199000300E8227A1EC0AF0ADC500F101010F0E57
:1019A0000101001724EC1FF033C182F40401300E52
:1019B0008227A1EC0AF004013A0E826FA1EC0AF032
:1019C000ACC500F10101003B0F0E001724EC1FF025
:1019D00033C182F40401300E8227A1EC0AF0ACC5B9
:1019E00000F101010F0E0101001724EC1FF033C1BB
:1019F00082F40401300E8227A1EC0AF004013A0EB1
:101A0000826FA1EC0AF0ABC500F10101003B0F0EA3
:101A1000001724EC1FF033C182F40401300E82273A
:101A2000A1EC0AF0ABC500F101010F0E001724EC88
:101A30001FF033C182F40401300E8227A1EC0AF0BA
:101A4000120084C3E8FF0F0BE83AE8CFB1F585C375
:101A5000E8FF0F0B0501B11387C3E8FF0F0BE83A4E
:101A6000E8CFB0F588C3E8FF0F0B0501B0138AC3B8
:101A7000E8FF0F0BE83AE8CFAFF58BC3E8FF0F0B99
:101A80000501AF138DC3E8FF0F0BE8CFAEF58FC391
:101A9000E8FF0F0BE83AE8CFADF590C3E8FF0F0B76
:101AA0000501AD1392C3E8FF0F0BE83AE8CFACF5A0
:101AB00093C3E8FF0F0B0501AC1395C3E8FF0F0BB1
:101AC000E83AE8CFABF596C3E8FF0F0B0501AB137F
:101AD0004EEC20F004014C0E826FA1EC0AF00401E0
:101AE000430E826FA1EC0AF033EF0CF021EC26F0EC
:101AF00081EC1FF02DC500F124EC1FF004014C0E09
:101B0000826FA1EC0AF00401300E826FA1EC0AF0A2
:101B100004012C0E826FA1EC0AF031C182F40401A1
:101B2000300E8227A1EC0AF032C182F40401300E9B
:101B30008227A1EC0AF033C182F40401300E82271F
:101B4000A1EC0AF004012C0E826FA1EC0AF081ECEA
:101B50001FF02EC500F124EC1FF031C182F4040106
:101B6000300E8227A1EC0AF032C182F40401300E5B
:101B70008227A1EC0AF033C182F40401300E8227DF
:101B8000A1EC0AF0D5EF10F004014C0E826FA1EC2D
:101B90000AF00401650E826FA1EC0AF02EEC22F02F
:101BA000D5EF10F004014C0E826FA1EC0AF0040195
:101BB000450E826FA1EC0AF04BEC22F0D5EF10F04D
:101BC00004014C0E826FA1EC0AF00401620E826FD8
:101BD000A1EC0AF085EC22F0D5EF10F004014C0ED8
:101BE000826FA1EC0AF00401420E826FA1EC0AF0B0
:101BF00068EC22F0D5EF10F004014C0E826FA1ECDE
:101C00000AF004015A0E826FA1EC0AF004012C0EB6
:101C1000826FA1EC0AF021EC26F081EC1FF00501A7
:101C20002E51130A06E005012E51170A0DE02DEF83
:101C30000EF00101000E006F000E016F100E026F1A
:101C4000000E036F2DEF0EF00101000E006F000E6D
:101C5000016F000E026F010E036F0101100E046F81
:101C6000000E056F000E066F000E076FB7EC1EF03A
:101C700024EC1FF02AC182F40401300E8227A1EC6B
:101C80000AF02BC182F40401300E8227A1EC0AF085
:101C90002CC182F40401300E8227A1EC0AF02DC180
:101CA00082F40401300E8227A1EC0AF02EC182F4E6
:101CB0000401300E8227A1EC0AF02FC182F4040146
:101CC000300E8227A1EC0AF030C182F40401300EFC
:101CD0008227A1EC0AF031C182F40401300E822780
:101CE000A1EC0AF032C182F40401300E8227A1EC8B
:101CF0000AF033C182F40401300E8227A1EC0AF00D
:101D0000D5EF10F004014C0E826FA1EC0AF0040133
:101D1000310E826FA1EC0AF004012C0E826FA1EC4F
:101D20000AF025C500F126C501F127C502F128C535
:101D300003F10101100E046F000E056F000E066F17
:101D4000000E076FB7EC1EF024EC1FF02AC182F4DE
:101D50000401300E8227A1EC0AF02BC182F40401A9
:101D6000300E8227A1EC0AF02CC182F40401300E5F
:101D70008227A1EC0AF02DC182F40401300E8227E3
:101D8000A1EC0AF02EC182F40401300E8227A1ECEE
:101D90000AF02FC182F40401300E8227A1EC0AF070
:101DA00030C182F40401300E8227A1EC0AF031C167
:101DB00082F40401300E8227A1EC0AF032C182F4D1
:101DC0000401300E8227A1EC0AF033C182F4040131
:101DD000300E8227A1EC0AF0D5EF10F004014C0E72
:101DE000826FA1EC0AF00401320E826FA1EC0AF0BE
:101DF0007BEC24F0D5EF10F004014C0E826FA1ECC7
:101E00000AF00401330E826FA1EC0AF0D8EC24F042
:101E10008CEF0EF004014C0E826FA1EC0AF004016D
:101E2000340E826FA1EC0AF004012C0E826FA1EC3B
:101E30000AF0C2EC1FF084C32AF185C32BF186C3DC
:101E40002CF187C32DF188C32EF189C32FF18AC3EA
:101E500030F18BC331F18CC332F18DC333F1010109
:101E6000296BCFEC1FF046EC1FF0100E046F000E34
:101E7000056F000E066F000E076F97EC1EF000C195
:101E800021F501C122F502C123F503C124F5D4ECEB
:101E900025F034C5ABF535C5ACF536C5ADF537C560
:101EA000AEF538C5AFF539C5B0F53AC5B1F53EEC7C
:101EB0000CF004012C0E826FA1EC0AF03BC500F17E
:101EC0003CC501F13DC502F13EC503F10101000E23
:101ED000046F000E056F010E066F000E076FB7EC62
:101EE0001EF024EC1FF0296778EF0FF07DEF0FF064
:101EF00004012D0E826FA1EC0AF030C182F40401BE
:101F0000300E8227A1EC0AF031C182F40401300EB8
:101F10008227A1EC0AF004012E0E826FA1EC0AF0D8
:101F200032C182F40401300E8227A1EC0AF033C1E1
:101F300082F40401300E8227A1EC0AF004012C0E79
:101F4000826FA1EC0AF081EC1FF03FC500F140C5A3
:101F500001F1EAEC19F004012C0E826FA1EC0AF0F9
:101F600081EC1FF041C500F124EC1FF031C182F477
:101F70000401300E8227A1EC0AF032C182F4040180
:101F8000300E8227A1EC0AF033C182F40401300E36
:101F90008227A1EC0AF0D5EF10F0C2EC1FF085C348
:101FA0002AF186C32BF187C32CF188C32DF189C395
:101FB0002EF18AC32FF18BC330F18CC331F18DC365
:101FC00032F18EC333F10101296BCFEC1FF046ECE7
:101FD0001FF00101010E046F000E056F000E066F69
:101FE000000E076F86EC1EF0100E046F000E056FDA
:101FF000000E066F000E076F97EC1EF000C129F56A
:1020000001C12AF502C12BF503C12CF504EC24F023
:1020100004014C0E826FA1EC0AF00401460E826F9F
:10202000A1EC0AF004012C0E826FA1EC0AF025C588
:1020300000F126C501F127C502F128C503F1010110
:10204000100E046F000E056F000E066F000E076F76
:10205000B7EC1EF024EC1FF02AC182F40401300E0C
:102060008227A1EC0AF02BC182F40401300E8227F2
:10207000A1EC0AF02CC182F40401300E8227A1ECFD
:102080000AF02DC182F40401300E8227A1EC0AF07F
:102090002EC182F40401300E8227A1EC0AF02FC178
:1020A00082F40401300E8227A1EC0AF030C182F4E0
:1020B0000401300E8227A1EC0AF031C182F4040140
:1020C000300E8227A1EC0AF032C182F40401300EF6
:1020D0008227A1EC0AF033C182F40401300E82277A
:1020E000A1EC0AF0D5EF10F00F98D8EC24F0C0EF77
:1020F00018F004014C0E826FA1EC0AF00401350EB9
:10210000826FA1EC0AF004012C0E826FA1EC0AF0A0
:1021100081EC1FF00784B5C500F1079424EC1FF093
:1021200031C182F40401300E8227A1EC0AF032C1E1
:1021300082F40401300E8227A1EC0AF033C182F44C
:102140000401300E8227A1EC0AF0D5EF10F09BECD1
:1021500024F081EC1FF033C500F124EC1FF00401E2
:102160004C0E826FA1EC0AF00401360E826FA1ECD6
:102170000AF004012C0E826FA1EC0AF031C182F446
:102180000401300E8227A1EC0AF032C182F404016E
:10219000300E8227A1EC0AF033C182F40401300E24
:1021A0008227A1EC0AF0D5EF10F0ABEC0AF0C0EFFB
:1021B00018F004014C0E826FA1EC0AF00401500EDD
:1021C000826FA1EC0AF004012C0E826FA1EC0AF0E0
:1021D00085C32AF186C32BF187C32CF188C32DF167
:1021E00089C32EF18AC32FF18BC330F18CC331F137
:1021F0008DC332F18EC333F10101CFEC1FF046ECF9
:102200001FF003018451530A0DE0030184514D0A6C
:1022100038E00401780E826FA1EC0AF0ABEC0AF012
:10222000C0EF18F00401530E826FA1EC0AF0250EE6
:102230000C6E00C10BF09CEC07F0260E0C6E01C179
:102240000BF09CEC07F0270E0C6E02C10BF09CEC1F
:1022500007F0280E0C6E03C10BF09CEC07F000C1D8
:1022600053F501C154F502C155F503C156F500C13E
:1022700057F501C158F502C159F503C15AF5B6EF3A
:1022800011F004014D0E826FA1EC0AF0290E0C6EC4
:1022900000C10BF09CEC07F000C15BF500C15CF5E0
:1022A000B6EF11F004014C0E826FA1EC0AF00401AC
:1022B000540E826FA1EC0AF004012C0E826FA1EC87
:1022C0000AF084C32AF185C32BF186C32CF187C39E
:1022D0002DF188C32EF189C32FF18AC330F18BC34E
:1022E00031F18DC332F18EC333F10101CFEC1FF018
:1022F00046EC1FF00101000E046F000E056F010E89
:10230000066F000E076F97EC1EF0210E0C6E00C1D9
:102310000BF09CEC07F0220E0C6E01C10BF09CEC54
:1023200007F0230E0C6E02C10BF09CEC07F0240E9C
:102330000C6E03C10BF09CEC07F000C15DF501C110
:102340005EF502C15FF503C160F5B6EF11F004015F
:102350004C0E826FA1EC0AF00401490E826FA1ECD1
:102360000AF004012C0E826FA1EC0AF0250EB3ECEA
:1023700007F0E8CF00F1260EB3EC07F0E8CF01F14B
:10238000270EB3EC07F0E8CF02F1280EB3EC07F00C
:10239000E8CF03F124EC1FF007EC1DF00401730EED
:1023A000826FA1EC0AF004012C0E826FA1EC0AF0FE
:1023B00081EC1FF0290EB3EC07F0E8CF00F124EC1C
:1023C0001FF007EC1DF00401730E826FA1EC0AF000
:1023D00004012C0E826FA1EC0AF057C500F158C51C
:1023E00001F159C502F15AC503F124EC1FF007ECC5
:1023F0001DF00401730E826FA1EC0AF004012C0E93
:10240000826FA1EC0AF081EC1FF05CC500F124ECB6
:102410001FF007EC1DF004016D0E826FA1EC0AF0B5
:1024200004012C0E826FA1EC0AF05DC500F15EC5BF
:1024300001F15FC502F160C503F1DBEC18F00401A6
:102440002C0E826FA1EC0AF0ABEC0AF0C0EF18F092
:1024500083C32AF184C32BF185C32CF186C32DF1EC
:1024600087C32EF188C32FF189C330F18AC331F1BC
:102470008BC332F18CC333F10101CFEC1FF046EC7A
:102480001FF0160E0C6E00C10BF09CEC07F0170E3F
:102490000C6E01C10BF09CEC07F0180E0C6E02C123
:1024A0000BF09CEC07F0190E0C6E03C10BF09CECCA
:1024B00007F000C18AF101C18BF102C18CF103C1A7
:1024C0008DF100C18EF101C18FF102C190F103C104
:1024D00091F10AEF13F083C32AF184C32BF185C372
:1024E0002CF186C32DF187C32EF188C32FF189C348
:1024F00030F18AC331F18BC332F18CC333F1010166
:10250000CFEC1FF046EC1FF000C18AF101C18BF146
:1025100002C18CF103C18DF100C18EF101C18FF1B7
:1025200002C190F103C191F10AEF13F083C32AF1C4
:1025300084C32BF185C32CF186C32DF187C32EF103
:1025400088C32FF189C330F18AC331F18CC332F1D2
:102550008DC333F10101CFEC1FF046EC1FF00101F8
:10256000000E046F000E056F010E066F000E076F60
:1025700097EC1EF01A0E0C6E00C10BF09CEC07F0ED
:102580001B0E0C6E01C10BF09CEC07F01C0E0C6EC8
:1025900002C10BF09CEC07F01D0E0C6E03C10BF09A
:1025A0009CEC07F000C192F101C193F102C194F1DA
:1025B00003C195F10AEF13F083C32AF184C32BF111
:1025C00085C32CF186C32DF187C32EF188C32FF16B
:1025D00089C330F18AC331F18CC332F18DC333F139
:1025E0000101CFEC1FF046EC1FF00101000E046F5B
:1025F000000E056F010E066F000E076F97EC1EF0C0
:1026000000C192F101C193F102C194F103C195F1AE
:102610000AEF13F0160EB3EC07F0E8CF00F1170E37
:10262000B3EC07F0E8CF01F1180EB3EC07F0E8CFF8
:1026300002F1190EB3EC07F0E8CF03F124EC1FF020
:1026400007EC1DF00401730E826FA1EC0AF0040187
:102650002C0E826FA1EC0AF08AC100F18BC101F14E
:102660008CC102F18DC103F124EC1FF007EC1DF0C9
:102670000401730E826FA1EC0AF004012C0E826F2C
:10268000A1EC0AF01A0EB3EC07F0E8CF00F11B0E34
:10269000B3EC07F0E8CF01F11C0EB3EC07F0E8CF84
:1026A00002F11D0EB3EC07F0E8CF03F1DBEC18F0FC
:1026B00004012C0E826FA1EC0AF092C100F193C1CB
:1026C00001F194C102F195C103F1DBEC18F0ABEC20
:1026D0000AF0C0EF18F00401690E826FA1EC0AF055
:1026E00004012C0E826FA1EC0AF00101040E006FB0
:1026F000000E016F000E026F000E036F24EC1FF03E
:102700002CC182F40401300E8227A1EC0AF02DC105
:1027100082F40401300E8227A1EC0AF02EC182F46B
:102720000401300E8227A1EC0AF02FC182F40401CB
:10273000300E8227A1EC0AF030C182F40401300E81
:102740008227A1EC0AF031C182F40401300E822705
:10275000A1EC0AF032C182F40401300E8227A1EC10
:102760000AF033C182F40401300E8227A1EC0AF092
:1027700004012C0E826FA1EC0AF00101060E006F1D
:10278000000E016F000E026F000E036F24EC1FF0AD
:102790002CC182F40401300E8227A1EC0AF02DC175
:1027A00082F40401300E8227A1EC0AF02EC182F4DB
:1027B0000401300E8227A1EC0AF02FC182F404013B
:1027C000300E8227A1EC0AF030C182F40401300EF1
:1027D0008227A1EC0AF031C182F40401300E822775
:1027E000A1EC0AF032C182F40401300E8227A1EC80
:1027F0000AF033C182F40401300E8227A1EC0AF002
:1028000004012C0E826FA1EC0AF001011E0E006F74
:10281000000E016F000E026F000E036F24EC1FF01C
:102820002CC182F40401300E8227A1EC0AF02DC1E4
:1028300082F40401300E8227A1EC0AF02EC182F44A
:102840000401300E8227A1EC0AF02FC182F40401AA
:10285000300E8227A1EC0AF030C182F40401300E60
:102860008227A1EC0AF031C182F40401300E8227E4
:10287000A1EC0AF032C182F40401300E8227A1ECEF
:102880000AF033C182F40401300E8227A1EC0AF071
:1028900004012C0E826FA1EC0AF0200EF86EF76A8C
:1028A000F66A04010900F5CF82F4A1EC0AF00900F0
:1028B000F5CF82F4A1EC0AF00900F5CF82F4A1EC87
:1028C0000AF00900F5CF82F4A1EC0AF00900F5CF77
:1028D00082F4A1EC0AF00900F5CF82F4A1EC0AF031
:1028E0000900F5CF82F4A1EC0AF00900F5CF82F4DB
:1028F000A1EC0AF0ABEC0AF0C0EF18F08351630AC8
:10290000D8A4C0EF18F08451610AD8A4C0EF18F021
:1029100085516C0AD8A4C0EF18F08651410A42E0F4
:102920008651440A1BE08651420AD8B4E5EF14F000
:102930008651350AD8B44AEF1AF08651360AD8B40F
:102940009FEF1AF08651370AD8B408EF1BF0865172
:10295000380AD8B466EF1BF0C0EF18F00798079A52
:1029600004017A0E826FA1EC0AF00401780E826FE6
:10297000A1EC0AF00401640E826FA1EC0AF081A8B8
:10298000C9EF14F00401550E826FA1EC0AF0CEEFEE
:1029900014F004014C0E826FA1EC0AF0ABEC0AF0CB
:1029A000C0EF18F00788079A04017A0E826FA1EC35
:1029B0000AF00401410E826FA1EC0AF00401610EDD
:1029C000826FA1EC0AF0BFEF14F00798078A0401A8
:1029D0007A0E826FA1EC0AF00401420E826FA1EC24
:1029E0000AF00401610E826FA1EC0AF0BFEF14F04F
:1029F0000101666703EF15F0676703EF15F068677D
:102A000003EF15F069671BEF15F04F670FEF15F037
:102A100050670FEF15F051670FEF15F052671BEF7E
:102A200015F00101000E006F000E016F000E026F25
:102A3000000E036F12000101620E046F010E056F9C
:102A4000000E066F000E076F66C100F167C101F14D
:102A500068C102F169C103F186EC1EF003BF9FEF6C
:102A600015F00101000E046FA80E056F550E066FDC
:102A7000020E076F66C100F167C101F168C102F182
:102A800069C103F166C186F167C187F168C188F148
:102A900069C189F186EC1EF003BF58EF15F0010102
:102AA000000E866FA80E876F550E886F020E896F15
:102AB0000E0EB3EC07F0E8CF18F10F0EB3EC07F0F1
:102AC000E8CF19F1100EB3EC07F0E8CF1AF1110EB0
:102AD000B3EC07F0E8CF1BF1CFEC1DF086C104F199
:102AE00087C105F188C106F189C107F186EC1EF0A6
:102AF000078293EC1DF0CFEC1DF0079293EC1DF0D4
:102B000086C100F187C101F188C102F189C103F1D9
:102B1000079293EC1DF0CC0E046FE00E056F870E4C
:102B2000066F050E076F86EC1EF000C118F101C19B
:102B300019F102C11AF103C11BF1D7EF15F0010120
:102B4000800E006F1A0E016F060E026F000E036FEB
:102B50004FC104F150C105F151C106F152C107F155
:102B600086EC1EF003AFB8EF15F081EC1FF01200F9
:102B70000E0EB3EC07F0E8CF18F10F0EB3EC07F030
:102B8000E8CF19F1100EB3EC07F0E8CF1AF1110EEF
:102B9000B3EC07F0E8CF1BF14FC100F150C101F1D8
:102BA00051C102F152C103F1078293EC1DF018C12B
:102BB00000F119C101F11AC102F11BC103F11200A8
:102BC0000401730E826FA1EC0AF004012C0E826FD7
:102BD000A1EC0AF0078462C166F163C167F164C1C8
:102BE00068F165C169F14BC14FF14CC150F14DC164
:102BF00051F14EC152F157C159F158C15AF10794E0
:102C000006EC16F0ABEC0AF0C0EF18F066C100F16C
:102C100067C101F168C102F169C103F1010124EC4E
:102C20001FF007EC1DF00401630E826FA1EC0AF0A7
:102C300004012C0E826FA1EC0AF04FC100F150C1CB
:102C400001F151C102F152C103F1010124EC1FF065
:102C500007EC1DF00401660E826FA1EC0AF004017E
:102C60002C0E826FA1EC0AF081EC1FF059C100F12B
:102C70005AC101F1010124EC1FF007EC1DF0040121
:102C8000740E826FA1EC0AF0120010820401530E40
:102C9000826FA1EC0AF004012C0E826FA1EC0AF005
:102CA00083C32AF184C32BF185C32CF186C32DF194
:102CB00087C32EF188C32FF189C330F18AC331F164
:102CC0008BC332F18CC333F10101CFEC1FF046EC22
:102CD0001FF000C166F101C167F102C168F103C1D3
:102CE00069F18EC32AF18FC32BF190C32CF191C3EC
:102CF0002DF192C32EF193C32FF194C330F195C3FC
:102D000031F196C332F197C333F10101CFEC1FF0DB
:102D100046EC1FF000C14FF101C150F102C151F169
:102D200003C152F1C2EC1FF099C32FF19AC330F1E5
:102D30009BC331F19CC332F19DC333F10101CFEC50
:102D40001FF046EC1FF000C159F101C15AF106EC29
:102D500016F004012C0E826FA1EC0AF0B7EF16F00A
:102D60008251520A03E10F82B7EF16F00F9282519F
:102D7000750A03E11084BEEF16F010948251550AD3
:102D800003E11086C5EF16F01096078410B222EF0B
:102D900017F010A40EEF17F0B6C166F1B7C167F1D6
:102DA000B8C168F1B9C169F1BAC16AF1BBC16BF1CF
:102DB000BCC16CF1BDC16DF1BEC16EF1BFC16FF19F
:102DC000C0C170F1C1C171F1C2C172F1C3C173F16F
:102DD000C4C174F1C5C175F1C6C176F1C7C177F13F
:102DE000C8C178F1C9C179F1CAC17AF1CBC17BF10F
:102DF000CCC17CF1CDC17DF1CEC17EF1CFC17FF1DF
:102E0000D0C180F1D1C181F1D2C182F1D3C183F1AE
:102E1000D4C184F1D5C185F116EF17F062C166F116
:102E200063C167F164C168F165C169F14BC14FF1DC
:102E30004CC150F14DC151F14EC152F157C159F140
:102E400058C15AF107940FA044EF17F0010192679F
:102E500031EF17F0936731EF17F0946731EF17F008
:102E6000956735EF17F044EF17F0F8EC14F092C1C6
:102E700004F193C105F194C106F195C107F186EC07
:102E80001EF003BF88EF18F0F8EC14F00101000EFB
:102E9000046F000E056F010E066F000E076FB7EC92
:102EA0001EF010A45BEF17F00401750E826FA1EC09
:102EB0000AF060EF17F00401720E826FA1EC0AF0C5
:102EC00004012C0E826FA1EC0AF024EC1FF029679C
:102ED0006FEF17F00401200E826F72EF17F00401FC
:102EE0002D0E826FA1EC0AF030C182F40401300E85
:102EF0008227A1EC0AF031C182F40401300E82274E
:102F0000A1EC0AF004012E0E826FA1EC0AF032C18E
:102F100082F40401300E8227A1EC0AF033C182F45E
:102F20000401300E8227A1EC0AF004016D0E826FBD
:102F3000A1EC0AF004012C0E826FA1EC0AF04FC143
:102F400000F150C101F151C102F152C103F101017F
:102F500024EC1FF007EC1DF00401480E826FA1EC79
:102F60000AF004017A0E826FA1EC0AF004012C0E23
:102F7000826FA1EC0AF066C100F167C101F168C17E
:102F800002F169C103F1010124EC1FF007EC1DF00F
:102F90000401630E826FA1EC0AF004012C0E826F13
:102FA000A1EC0AF066C100F167C101F168C102F14C
:102FB00069C103F101010A0E046F000E056F000ED6
:102FC000066F000E076F97EC1EF0000E046F120ED6
:102FD000056F000E066F000E076FB7EC1EF024ECB5
:102FE0001FF02AC182F40401300E8227A1EC0AF0FE
:102FF0002BC182F40401300E8227A1EC0AF02CC10F
:1030000082F40401300E8227A1EC0AF02DC182F473
:103010000401300E8227A1EC0AF02EC182F40401D3
:10302000300E8227A1EC0AF02FC182F40401300E89
:103030008227A1EC0AF030C182F40401300E82270D
:10304000A1EC0AF004012E0E826FA1EC0AF031C14E
:1030500082F40401300E8227A1EC0AF032C182F41E
:103060000401300E8227A1EC0AF033C182F404017E
:10307000300E8227A1EC0AF00401730E826FA1ECDE
:103080000AF004012C0E826FA1EC0AF081EC1FF013
:1030900059C100F15AC101F1EAEC19F00FB254EF35
:1030A00018F00FA086EF18F004012C0E826FA1EC2F
:1030B0000AF0200EF86EF76AF66A04010900F5CFEF
:1030C00082F4A1EC0AF00900F5CF82F4A1EC0AF039
:1030D0000900F5CF82F4A1EC0AF00900F5CF82F4E3
:1030E000A1EC0AF00900F5CF82F4A1EC0AF0090086
:1030F000F5CF82F4A1EC0AF00900F5CF82F4A1EC3F
:103100000AF00900F5CF82F4A1EC0AF0ABEC0AF06A
:103110000F90C0EF18F00401630E826FA1EC0AF06B
:1031200004012C0E826FA1EC0AF0C6EC18F0040129
:103130002C0E826FA1EC0AF039EC19F004012C0E70
:10314000826FA1EC0AF0B5EC19F004012C0E826F2D
:10315000A1EC0AF00101F80E006FCD0E016F660EB2
:10316000026F030E036FDBEC18F004012C0E826F6C
:10317000A1EC0AF0CBEC19F0ABEC0AF0C0EF18F0C0
:103180000301C26B07901092CFEF1BF0D8900E0E88
:10319000B3EC07F0E8CF00F10F0EB3EC07F0E8CF87
:1031A00001F1100EB3EC07F0E8CF02F1110EB3EC11
:1031B00007F0E8CF03F10101000E046F000E056F68
:1031C000010E066F000E076FB7EC1EF024EC1FF027
:1031D0002AC182F40401300E8227A1EC0AF02BC12F
:1031E00082F40401300E8227A1EC0AF02CC182F493
:1031F0000401300E8227A1EC0AF02DC182F40401F3
:10320000300E8227A1EC0AF02EC182F40401300EA8
:103210008227A1EC0AF02FC182F40401300E82272C
:10322000A1EC0AF030C182F40401300E8227A1EC37
:103230000AF031C182F40401300E8227A1EC0AF0B9
:1032400004012E0E826FA1EC0AF032C182F4040157
:10325000300E8227A1EC0AF033C182F40401300E53
:103260008227A1EC0AF004016D0E826FA1EC0AF036
:103270001200120EB3EC07F0E8CF00F1130EB3EC1E
:1032800007F0E8CF01F1140EB3EC07F0E8CF02F13C
:10329000150EB3EC07F0E8CF03F101010A0E046F3D
:1032A000000E056F000E066F000E076F97EC1EF004
:1032B000000E046F120E056F000E066F000E076FF2
:1032C000B7EC1EF024EC1FF02AC182F40401300E8A
:1032D0008227A1EC0AF02BC182F40401300E822770
:1032E000A1EC0AF02CC182F40401300E8227A1EC7B
:1032F0000AF02DC182F40401300E8227A1EC0AF0FD
:103300002EC182F40401300E8227A1EC0AF02FC1F5
:1033100082F40401300E8227A1EC0AF030C182F45D
:103320000401300E8227A1EC0AF004012E0E826FF8
:10333000A1EC0AF031C182F40401300E8227A1EC25
:103340000AF032C182F40401300E8227A1EC0AF0A7
:1033500033C182F40401300E8227A1EC0AF004018B
:10336000730E826FA1EC0AF012000A0EB3EC07F0A4
:10337000E8CF00F10B0EB3EC07F0E8CF01F10C0E33
:10338000B3EC07F0E8CF02F10D0EB3EC07F0E8CF95
:1033900003F1EAEF19F0060EB3EC07F0E8CF00F105
:1033A000070EB3EC07F0E8CF01F1080EB3EC07F01D
:1033B000E8CF02F1090EB3EC07F0E8CF03F1EAEF32
:1033C00019F0010181EC1FF0078457C100F158C1C9
:1033D00001F107940101E80E046F800E056F000EE5
:1033E000066F000E076F97EC1EF0000E046F040EC0
:1033F000056F000E066F000E076FB7EC1EF0880E0B
:10340000046F130E056F000E066F000E076F86EC3B
:103410001EF00A0E046F000E056F000E066F000E00
:10342000076FB7EC1EF024EC1FF0010129671EEFB7
:103430001AF00401200E826F21EF1AF004012D0E04
:10344000826FA1EC0AF030C182F40401300E8227B1
:10345000A1EC0AF031C182F40401300E8227A1EC04
:103460000AF032C182F40401300E8227A1EC0AF086
:1034700004012E0E826FA1EC0AF033C182F4040124
:10348000300E8227A1EC0AF00401430E826FA1ECFA
:103490000AF0120087C32AF188C32BF189C32CF1EB
:1034A0008AC32DF18BC32EF18CC32FF18DC330F164
:1034B0008EC331F190C332F191C333F10101296B15
:1034C000CFEC1FF046EC1FF00101000E046F000E60
:1034D000056F010E066F000E076F97EC1EF00E0EC3
:1034E0000C6E00C10BF09CEC07F00F0E0C6E01C1CE
:1034F0000BF09CEC07F0100E0C6E02C10BF09CEC74
:1035000007F0110E0C6E03C10BF09CEC07F00401E8
:103510007A0E826FA1EC0AF004012C0E826FA1ECEE
:103520000AF00401350E826FA1EC0AF004012C0EA2
:10353000826FA1EC0AF0C6EC18F0CEEF14F087C34E
:103540002AF188C32BF189C32CF18AC32DF18BC3D7
:103550002EF18CC32FF18DC330F18EC331F190C3A6
:1035600032F191C333F10101296BCFEC1FF046EC2E
:103570001FF0880E046F130E056F000E066F000E0D
:10358000076F8BEC1EF0000E046F040E056F000E2B
:10359000066F000E076F97EC1EF00101E80E046F36
:1035A000800E056F000E066F000E076FB7EC1EF061
:1035B0000A0E0C6E00C10BF09CEC07F00B0E0C6EAB
:1035C00001C10BF09CEC07F00C0E0C6E02C10BF06D
:1035D0009CEC07F00D0E0C6E03C10BF09CEC07F099
:1035E00004017A0E826FA1EC0AF004012C0E826FA6
:1035F000A1EC0AF00401360E826FA1EC0AF004017E
:103600002C0E826FA1EC0AF0B5EC19F0CEEF14F09D
:1036100087C32AF188C32BF189C32CF18AC32DF10A
:103620008BC32EF18CC32FF18DC330F18FC331F1D9
:1036300090C332F191C333F10101CFEC1FF046EC9E
:103640001FF0000E046F120E056F000E066F000EC5
:10365000076F97EC1EF001010A0E046F000E056F54
:10366000000E066F000E076FB7EC1EF0120E0C6E08
:1036700000C10BF09CEC07F0130E0C6E01C10BF0B7
:103680009CEC07F0140E0C6E02C10BF09CEC07F0E2
:10369000150E0C6E03C10BF09CEC07F004017A0EC2
:1036A000826FA1EC0AF004012C0E826FA1EC0AF0EB
:1036B0000401370E826FA1EC0AF004012C0E826F18
:1036C000A1EC0AF039EC19F0CEEF14F087C32AF11F
:1036D00088C32BF189C32CF18AC32DF18BC32EF142
:1036E0008CC32FF18DC330F18EC331F190C332F111
:1036F00091C333F10101296BCFEC1FF046EC1FF0B1
:10370000880E046F130E056F000E066F000E076F14
:103710008BEC1EF0000E046F040E056F000E066F9A
:10372000000E076F97EC1EF00101E80E046F800E8B
:10373000056F000E066F000E076FB7EC1EF0060E49
:103740000C6E00C10BF09CEC07F0070E0C6E01C173
:103750000BF09CEC07F0080E0C6E02C10BF09CEC19
:1037600007F0090E0C6E03C10BF09CEC07F004018E
:103770007A0E826FA1EC0AF004012C0E826FA1EC8C
:103780000AF00401380E826FA1EC0AF004012C0E3D
:10379000826FA1EC0AF0CBEC19F0CEEF14F081A807
:1037A0008DEF1CF007A846EF1CF00101800E006FA2
:1037B0001A0E016F060E026F000E036F4BC104F16B
:1037C0004CC105F14DC106F14EC107F186EC1EF06A
:1037D00003BF8DEF1CF001EC1DF04BC100F14CC19B
:1037E00001F14DC102F14EC103F1078293EC1DF0CE
:1037F00018C104F119C105F11AC106F11BC107F185
:10380000F80E006FCD0E016F660E026F030E036F90
:1038100086EC1EF00E0E0C6E00C10BF09CEC07F057
:103820000F0E0C6E01C10BF09CEC07F0100E0C6E2D
:1038300002C10BF09CEC07F0110E0C6E03C10BF0F3
:103840009CEC07F00784010181EC1FF057C100F1E7
:1038500058C101F107940A0E0C6E00C10BF09CECEC
:1038600007F00B0E0C6E01C10BF09CEC07F00C0E78
:103870000C6E02C10BF09CEC07F00D0E0C6E03C138
:103880000BF09CEC07F007988DEF1CF007AA8DEF6A
:103890001CF00784010181EC1FF057C100F158C1F1
:1038A00001F10794060E0C6E00C10BF09CEC07F0C2
:1038B000070E0C6E01C10BF09CEC07F0080E0C6EAD
:1038C00002C10BF09CEC07F0090E0C6E03C10BF06B
:1038D0009CEC07F0078462C100F163C101F164C18F
:1038E00002F165C103F10794120E0C6E00C10BF0DA
:1038F0009CEC07F0130E0C6E01C10BF09CEC07F072
:10390000140E0C6E02C10BF09CEC07F0150E0C6E41
:1039100003C10BF09CEC07F0079A04018051811958
:103920007F0B0BE09EA809D014EE00F081517F0BB5
:10393000E126E750812B0F01AD6E05012F51010AE1
:1039400013E081AAB4EF1CF005012F51000A0AE030
:103950000FB8B4EF1CF005013067B4EF1CF00FB8DE
:10396000B4EF1CF060EF26F081B8C9EF1CF09FECBB
:1039700020F005012F51020A02E0C9EF1CF05C2F74
:10398000C9EF1CF05BC55CF50501010E306F3C0E04
:10399000316F0FEF0AF018C100F119C101F11AC11E
:1039A00002F11BC103F1000E046F000E056F010E42
:1039B000066F000E076FB7EC1EF029A1F6EF1CF0A2
:1039C0002051D8B4F6EF1CF018C100F119C101F173
:1039D0001AC102F11BC103F1000E046F000E056F46
:1039E0000A0E066F000E076FB7EC1EF01200010101
:1039F000045100130551011306510213075103131B
:103A000012000101186B196B1A6B1B6B12002AC193
:103A100082F40401300E8227A1EC0AF02BC182F45B
:103A20000401300E8227A1EC0AF02CC182F40401BB
:103A3000300E8227A1EC0AF02DC182F40401300E71
:103A40008227A1EC0AF02EC182F40401300E8227F5
:103A5000A1EC0AF02FC182F40401300E8227A1EC00
:103A60000AF030C182F40401300E8227A1EC0AF082
:103A700031C182F40401300E8227A1EC0AF032C178
:103A800082F40401300E8227A1EC0AF033C182F4E3
:103A90000401300E8227A1EC0AF012002FC182F43B
:103AA0000401300E8227A1EC0AF030C182F4040137
:103AB000300E8227A1EC0AF031C182F40401300EED
:103AC0008227A1EC0AF032C182F40401300E822771
:103AD000A1EC0AF033C182F40401300E8227A1EC7C
:103AE0000AF01200060E116E060E126E060E136E0E
:103AF000112E78EF1DF0122E78EF1DF0132E78EFB7
:103B00001DF08B84020E116E020E126E020E136EE9
:103B1000112E88EF1DF0122E88EF1DF0132E88EF66
:103B20001DF08B9412000101005305E1015303E1E4
:103B3000025301E1002B56EC1EF081EC1FF03951CD
:103B4000006F3A51016F420E046F4B0E056F000E6D
:103B5000066F000E076F97EC1EF000C104F101C163
:103B600005F102C106F103C107F118C100F119C145
:103B700001F11AC102F11BC103F107B2C4EF1DF03C
:103B80008BEC1EF0C6EF1DF086EC1EF000C118F1A4
:103B900001C119F102C11AF103C11BF1120081EC3C
:103BA0001FF059C100F15AC101F1060EB3EC07F044
:103BB000E8CF04F1070EB3EC07F0E8CF05F1080EEB
:103BC000B3EC07F0E8CF06F1090EB3EC07F0E8CF4D
:103BD00007F186EC1EF000C124F101C125F102C1FC
:103BE00026F103C127F1290E046F000E056F000EA8
:103BF000066F000E076F97EC1EF0EE0E046F430E7B
:103C0000056F000E066F000E076F8BEC1EF024C1CF
:103C100004F125C105F126C106F127C107F197EC92
:103C20001EF000C11CF101C11DF102C11EF103C152
:103C30001FF1120EB3EC07F0E8CF04F1130EB3EC52
:103C400007F0E8CF05F1140EB3EC07F0E8CF06F16A
:103C5000150EB3EC07F0E8CF07F10D0E006F000E64
:103C6000016F000E026F000E036F97EC1EF0180E2E
:103C7000046F000E056F000E066F000E076FB7ECA5
:103C80001EF01CC104F11DC105F11EC106F11FC1CA
:103C900007F18BEC1EF06A0E046F2A0E056F000E02
:103CA000066F000E076F86EC1EF01200BF0EFA6E54
:103CB000200E3A6F396BD89000370137023703373F
:103CC000D8B067EF1EF03A2F5CEF1EF039073A07C5
:103CD0000353D8B412000331070B80093F6F033937
:103CE0000F0B010F396F80EC5FF0406F390580ECEE
:103CF0005FF0405D405F396B3F33D8B039273933CF
:103D00003FA97CEF1EF04051392712000101A6ECBB
:103D10001FF0D8B01200010103510719346F69EC8C
:103D20001FF0D8900751031934AF800F1200010122
:103D3000346B8DEC1FF0D8A0A3EC1FF0D8B01200AC
:103D400078EC1FF081EC1FF01F0E366FB9EC1FF0FE
:103D50000B35D8B069EC1FF0D8A00335D8B01200ED
:103D6000362FA6EF1EF034B190EC1FF012000101C7
:103D7000346B04510511061107110008D8A08DEC11
:103D80001FF0D8A0A3EC1FF0D8B01200086B096B8D
:103D90000A6B0B6BB9EC1FF01F0E366FB9EC1FF0FE
:103DA00007510B5DD8A4E1EF1EF006510A5DD8A4BF
:103DB000E1EF1EF00551095DD8A4E1EF1EF00451BA
:103DC000085DD8A0F4EF1EF00451085F0551D8A09B
:103DD000053D095F0651D8A0063D0A5F0751D8A0EE
:103DE000073D0B5FD8900081362FCEEF1EF034B127
:103DF00090EC1FF0346B8DEC1FF0D890BDEC1FF0F1
:103E000007510B5DD8A411EF1FF006510A5DD8A42D
:103E100011EF1FF00551095DD8A411EF1FF00451F7
:103E2000085DD8A020EF1FF0003F20EF1FF0013FFA
:103E300020EF1FF0023F20EF1FF0032BD8B4120039
:103E400034B190EC1FF012000101346B8DEC1FF0C7
:103E5000D8B01200C2EC1FF0200E366F00370137C9
:103E60000237033711EE33F00A0E376FE7360A0ECA
:103E7000E75CD8B0E76EE552372F36EF1FF0362FEC
:103E80002EEF1FF034B12981D890120001010A0EE3
:103E9000346F200E366F11EE29F03451376F0A0E51
:103EA000D890E652D8B0E726E732372F51EF1FF00F
:103EB0000333023301330033362F4BEF1FF0E7504B
:103EC000FF0FD8A00335D8B0120029B190EC1FF035
:103ED0001200045100270551D8B0053D01270651B5
:103EE000D8B0063D02270751D8B0073D032712007E
:103EF0000051086F0151096F02510A6F03510B6F96
:103F000012000101006B016B026B036B12000101D7
:103F1000046B056B066B076B12000335D8A012000B
:103F20000351800B001F011F021F031F003FA0EF62
:103F30001FF0013FA0EF1FF0023FA0EF1FF0032B87
:103F4000342B032512000735D8A012000751800B2F
:103F5000041F051F061F071F043FB6EF1FF0053F94
:103F6000B6EF1FF0063FB6EF1FF0072B342B0725E7
:103F700012000037013702370337083709370A378D
:103F80000B3712000101296B2A6B2B6B2C6B2D6BED
:103F90002E6B2F6B306B316B326B336B1200010168
:103FA0002A510F0B2A6F2B510F0B2B6F2C510F0B1C
:103FB0002C6F2D510F0B2D6F2E510F0B2E6F2F517C
:103FC0000F0B2F6F30510F0B306F31510F0B316FC3
:103FD00032510F0B326F33510F0B336F1200898444
:103FE000000EC76E220EC66E9E96C69E000EC96E4D
:103FF000FF0E9EB602D0E82EFCD79E96C69E000EFF
:10400000C96EFF0E9EB602D0E82EFCD7C9CFABF525
:104010009E96C69E000EC96EFF0E9EB602D0E82E7A
:10402000FCD7C9CFACF59E96C69E000EC96EFF0E9A
:104030009EB602D0E82EFCD7C9CFADF59E96C69E9F
:10404000000EC96EFF0E9EB602D0E82EFCD7C9CF77
:10405000AEF59E96C69E000EC96EFF0E9EB602D0AD
:10406000E82EFCD7C9CFAFF59E96C69E000EC96E4E
:10407000FF0E9EB602D0E82EFCD7C9CFB0F59E96B3
:10408000C69E000EC96EFF0E9EB602D0E82EFCD76B
:10409000C9CFB1F58994A2EC22F012008984000EF8
:1040A000C76E220EC66E9E96C69E800EC96EFF0E0D
:1040B0009EB602D0E82EFCD79E96C69EABC5C9FF21
:1040C000FF0E9EB602D0E82EFCD79E96C69EACC5CB
:1040D000C9FFFF0E9EB602D0E82EFCD79E96C69E64
:1040E000ADC5C9FFFF0E9EB602D0E82EFCD79E9646
:1040F000C69EAEC5C9FFFF0E9EB602D0E82EFCD705
:104100009E96C69EAFC5C9FFFF0E9EB602D0E82E92
:10411000FCD79E96C69EB0C5C9FFFF0E9EB602D0C4
:10412000E82EFCD79E96C69EB1C5C9FFFF0E9EB66F
:1041300002D0E82EFCD78994A2EC22F012008984E8
:10414000000EC76E220EC66E9E96C69E070EC96EE4
:10415000FF0E9EB602D0E82EFCD79E96C69E000E9D
:10416000C96EFF0E9EB602D0E82EFCD7C9CFABF5C4
:104170009E96C69E000EC96EFF0E9EB602D0E82E19
:10418000FCD7C9CFACF59E96C69E000EC96EFF0E39
:104190009EB602D0E82EFCD7C9CFADF59E96C69E3E
:1041A000000EC96EFF0E9EB602D0E82EFCD7C9CF16
:1041B000AEF58994A2EC22F08984000EC76E220E1F
:1041C000C66E9E96C69E0F0EC96EFF0E9EB602D09C
:1041D000E82EFCD79E96C69E000EC96EFF0E9EB6B8
:1041E00002D0E82EFCD7C9CFB3F58994A2EC22F017
:1041F00012008984000EC76E220EC66E9E96C69E61
:10420000870EC96EFF0E9EB602D0E82EFCD79E9692
:10421000C69EABC5C9FFFF0E9EB602D0E82EFCD7E6
:104220009E96C69EACC5C9FFFF0E9EB602D0E82E74
:10423000FCD79E96C69EADC5C9FFFF0E9EB602D0A6
:10424000E82EFCD79E96C69EAEC5C9FFFF0E9EB651
:1042500002D0E82EFCD78994A2EC22F089849E96A5
:10426000C69E8F0EC96EFF0E9EB602D0E82EFCD7FA
:104270009E96C69EB3C5C9FFFF0E9EB602D0E82E1D
:10428000FCD78994A2EC22F012008984000EC76E3C
:10429000220EC66E9E96C69E870EC96EFF0E9EB6F5
:1042A00002D0E82EFCD79E96C69E000EC96EFF0E69
:1042B0009EB602D0E82EFCD79E96C69E800EC96E92
:1042C000FF0E9EB602D0E82EFCD79E96C69E800EAC
:1042D000C96EFF0E9EB602D0E82EFCD79E96C69EF3
:1042E000800EC96EFF0E9EB602D0E82EFCD78994D0
:1042F000A2EC22F089849E96C69E8F0EC96EFF0E98
:104300009EB602D0E82EFCD79E96C69E010EC96EC0
:10431000FF0E9EB602D0E82EFCD78994A2EC22F0C4
:1043200012008984000EC76E220EC66E9E96C69E2F
:10433000870EC96EFF0E9EB602D0E82EFCD79E9661
:10434000C69E000EC96EFF0E9EB602D0E82EFCD7A8
:104350009E96C69E000EC96EFF0E9EB602D0E82E37
:10436000FCD79E96C69E800EC96EFF0E9EB602D0EA
:10437000E82EFCD79E96C69E800EC96EFF0E9EB696
:1043800002D0E82EFCD78994A2EC22F089849E9674
:10439000C69E8F0EC96EFF0E9EB602D0E82EFCD7C9
:1043A0009E96C69E010EC96EFF0E9EB602D0E82EE6
:1043B000FCD78994A2EC22F012008984000EC76E0B
:1043C000220EC66E9E96C69E8F0EC96EFF0E9EB6BC
:1043D00002D0E82EFCD7A2EC22F09E96C69E810E5B
:1043E000C96EFF0E9EB602D0E82EFCD78994A2ECCF
:1043F00022F08984000EC76E220EC66E9E96C69E5F
:104400008F0EC96EFF0E9EB602D0E82EFCD7A2EC2E
:1044100022F09E96C69E010EC96EFF0E9EB602D079
:10442000E82EFCD78994A2EC22F089849E96C69E41
:10443000910EC96EFF0E9EB602D0E82EFCD7A2ECFC
:1044400022F09E96C69EA50EC96EFF0E9EB602D0A5
:10445000E82EFCD78994A2EC22F012008984000E89
:10446000C76E220EC66E9E96C69E8F0EC96EFF0E3A
:104470009EB602D0E82EFCD7A2EC22F09E96C69EF5
:10448000810EC96EFF0E9EB602D0E82EFCD789942D
:10449000A2EC22F012008984000EC76E220EC66EB6
:1044A0009E96C69E8F0EC96EFF0E9EB602D0E82E57
:1044B000FCD7A2EC22F09E96C69E010EC96EFF0E9E
:1044C0009EB602D0E82EFCD78994A2EC22F012000E
:1044D0008984000EC76E220EC66E9E96C69E910EF1
:1044E000C96EFF0E9EB602D0E82EFCD7A2EC22F0D9
:1044F0009E96C69EA50EC96EFF0E9EB602D0E82EF1
:10450000FCD78994A2EC22F012008984000EC76EB9
:10451000220EC66E9E96C69E910EC96EFF0E9EB668
:1045200002D0E82EFCD7A2EC22F09E96C69E000E8A
:10453000C96EFF0E9EB602D0E82EFCD78994A2EC7D
:1045400022F01200050EE82EFED712000501256BA1
:10455000266B276B286B899A400EC76E200EC66E9D
:104560009E96C69E030EC96EFF0E9EB602D0E82E22
:10457000FCD79E96C69E27C5C9FFFF0E9EB602D0E9
:10458000E82EFCD79E96C69E26C5C9FFFF0E9EB696
:1045900002D0E82EFCD79E96C69E25C5C9FFFF0E09
:1045A0009EB602D0E82EFCD79E96C69EC952FF0E3C
:1045B0009EB602D0E82EFCD7898A0F01C950FF0AA7
:1045C00001E1120005012E51130A05E005012E51EB
:1045D000170A0CE012000501F00E256FFF0E266F82
:1045E0000F0E276F000E286FFFEF22F00501F00E6F
:1045F000256FFF0E266FFF0E276F000E286F899A1A
:10460000400EC76E200EC66E9E96C69E030EC96EE5
:10461000FF0E9EB602D0E82EFCD79E96C69E27C5FA
:10462000C9FFFF0E9EB602D0E82EFCD79E96C69E0E
:1046300026C5C9FFFF0E9EB602D0E82EFCD79E9677
:10464000C69E25C5C9FFFF0E9EB602D0E82EFCD738
:104650009E96C69EC952FF0E9EB602D0E82EFCD78B
:10466000898A0F01C950FF0A1DE005012E51130A66
:1046700005E005012E51170A0BE012000501000E9E
:10468000256F000E266F100E276F000E286F120088
:104690000501000E256F000E266F000E276F010E1C
:1046A000286F12000501256B266B276B286B05010F
:1046B0002E51130A05E005012E51170A0CE01200D5
:1046C0000501000E216F000E226F040E236F000EF5
:1046D000246F74EF23F00501000E216F000E226F8E
:1046E000800E236F000E246F21C500F122C501F159
:1046F00023C502F124C503F125C504F126C505F142
:1047000027C506F128C507F1F7EC1CF000C125F517
:1047100001C126F502C127F503C128F5899A400E8B
:10472000C76E200EC66E9E96C69E030EC96EFF0E05
:104730009EB602D0E82EFCD79E96C69E27C5C9FF1E
:10474000FF0E9EB602D0E82EFCD79E96C69E26C5CA
:10475000C9FFFF0E9EB602D0E82EFCD79E96C69EDD
:1047600025C5C9FFFF0E9EB602D0E82EFCD79E9647
:10477000C69EC952FF0E9EB602D0E82EFCD7898A8B
:10478000C950FF0A08E104C125F505C126F506C197
:1047900027F507C128F5D8900501243323332233A8
:1047A00021332151F00B216F2167DEEF23F02267C7
:1047B000DEEF23F02367DEEF23F0246774EF23F0AE
:1047C0000501100E2527E86A2623E86A2723E86AF0
:1047D00028231200E86A05012E51130A06E005019C
:1047E0002E51170A0BE0020E120005012851000A93
:1047F00003E12751F00B07E0010E120005012851DB
:10480000000A01E0010E120029C500F12AC501F1DC
:104810002BC502F12CC503F125C504F126C505F110
:1048200027C506F128C507F186EC1EF003BF12006C
:10483000EAEC23F05FE1899A400EC76E200EC66E47
:104840009E96C69E060EC96EFF0E9EB602D0E82E3C
:10485000FCD7898A899A9E96C69E020EC96EFF0E63
:104860009EB602D0E82EFCD79E96C69E27C5C9FFED
:10487000FF0E9EB602D0E82EFCD79E96C69E26C599
:10488000C9FFFF0E9EB602D0E82EFCD79E96C69EAC
:1048900025C5C9FFFF0E9EB602D0E82EFCD79E9616
:1048A000C69E000EC96EFF0E9EB602D0E82EFCD743
:1048B000898A899A9E96C69E050EC96EFF0E9EB67F
:1048C00002D0E82EFCD79E96C69EC952FF0E9EB619
:1048D00002D0E82EFCD7C9B063EF24F0898A050125
:1048E000100E2527E86A2623E86A2723E86A28238A
:1048F00004EF24F01200899A400EC76E200EC66E97
:104900009E96C69E060EC96EFF0E9EB602D0E82E7B
:10491000FCD7898A899A9E96C69EC70EC96EFF0EDD
:104920009EB602D0E82EFCD7898A0501256B266B3E
:10493000276B286B1200899A400EC76E200EC66E38
:104940009E96C69E050EC96EFF0E9EB602D0E82E3C
:10495000FCD79E96C69EC952FF0E9EB602D0E82E88
:10496000FCD7C9CF33F5898A1200899A400EC76EE9
:10497000200EC66E9E96C69EB90EC96EFF0E9EB6DE
:1049800002D0E82EFCD7898A1200899A400EC76EA1
:10499000200EC66E9E96C69EAB0EC96EFF0E9EB6CC
:1049A00002D0E82EFCD7898AFF0EE82EFED712002F
:1049B000EAEC23F0D8A41200899A400EC76E200EAC
:1049C000C66E9E96C69E030EC96EFF0E9EB602D0A0
:1049D000E82EFCD79E96C69E27C5C9FFFF0E9EB641
:1049E00002D0E82EFCD79E96C69E26C5C9FFFF0EB4
:1049F0009EB602D0E82EFCD79E96C69E25C5C9FF5E
:104A0000FF0E9EB602D0E82EFCD79E96C69EC952D7
:104A1000FF0E9EB602D0E82EFCD7898A0F01C9503E
:104A2000FF0AD8A4D3EF25F00501FE0E336FEFEC9B
:104A30001FF0ABC534F5ACC535F5ADC536F5AEC523
:104A400037F5AFC538F5B0C539F5B1C53AF50784C6
:104A5000B6C166F1B7C167F1B8C168F1B9C169F112
:104A60004BC14FF14CC150F14DC151F14EC152F10A
:104A700057C159F158C15AF1F8EC14F000C13BF597
:104A800001C13CF502C13DF503C13EF505015D677D
:104A900051EF25F05E6751EF25F05F6751EF25F08C
:104AA000606755EF25F062EF25F05DC504F15EC546
:104AB00005F15FC506F160C507F186EC1EF003BF86
:104AC000D3EF25F059C13FF55AC140F5B5C541F5C1
:104AD000B6C542F507940501100E326F899A400E53
:104AE000C76E200EC66E9E96C69E060EC96EFF0E3F
:104AF0009EB602D0E82EFCD7898A899A9E96C69ED9
:104B0000020EC96EFF0E9EB602D0E82EFCD79E960E
:104B1000C69E27C5C9FFFF0E9EB602D0E82EFCD761
:104B20009E96C69E26C5C9FFFF0E9EB602D0E82EF1
:104B3000FCD79E96C69E25C5C9FFFF0E9EB602D025
:104B4000E82EFCD725EE33F0322F02D0B3EF25F05C
:104B50009E96C69EDECFC9FFFF0E9EB602D0E82EFF
:104B6000FCD7A4EF25F0898A899A9E96C69E050EE9
:104B7000C96EFF0E9EB602D0E82EFCD79E96C69E4A
:104B8000C952FF0E9EB602D0E82EFCD7C9B0BEEFC8
:104B900025F0898A0501100E2527E86A2623E86A90
:104BA0002723E86A2823120021C500F122C501F15C
:104BB00023C502F124C503F1899A400EC76E200E69
:104BC000C66E9E96C69E0B0EC96EFF0E9EB602D096
:104BD000E82EFCD79E96C69E02C1C9FFFF0E9EB668
:104BE00002D0E82EFCD79E96C69E01C1C9FFFF0EDB
:104BF0009EB602D0E82EFCD79E96C69E00C1C9FF85
:104C0000FF0E9EB602D0E82EFCD79E96C69EC952D5
:104C1000FF0E9EB602D0E82EFCD725EE33F005013C
:104C2000100E326F9E96C69EC952FF0E9EB602D0DF
:104C3000E82EFCD7C9CFDEFF322F12EF26F0898A8B
:104C40001200899A400EC76E200EC66E9E96C69EB2
:104C5000900EC96EFF0E9EB602D0E82EFCD79E962F
:104C6000C69E000EC96EFF0E9EB602D0E82EFCD77F
:104C70009E96C69E000EC96EFF0E9EB602D0E82E0E
:104C8000FCD79E96C69E000EC96EFF0E9EB602D041
:104C9000E82EFCD79E96C69EC952FF0E9EB602D045
:104CA000E82EFCD7C9CF2DF59E96C69EC952FF0EA1
:104CB0009EB602D0E82EFCD7C9CF2EF5898A120005
:104CC00072EC1DF0B5C5E8FFD70802E372EC1DF0E9
:104CD000B5C5E8FFC80802E372EC1DF0B5C5E8FFF2
:104CE000B90802E372EC1DF0B5C5E8FFAA0802E3BB
:104CF00072EC1DF0B5C5E8FF9B0802E372EC1DF0F5
:104D00009FEC20F0B5EC24F0F29CF29E8B94C69AB6
:104D1000C2909482948C720ED36ED3A4FED78996DF
:104D20008A909390FF0EE8CF00F0E82EFED7002E79
:104D3000FCD78150F294F29A9E909D909E929D9203
:0E4D4000F298F292F290F286F28E0300FF00DB
:10BF0000E844F926000C160C2B0C3F0C520C640C68
:10BF1000760C860C960CA50CB30CC10CCF0CDC0C6B
:06BF2000E80CF40C000C1B
:00000001FF
